:1000000008308A000B2A0000FF00030E8301A100C4
:100010000A08A0008A010408A2007708A300780853
:10002000A4007908A5007A08A6007B08A70083131E
:1000300083120B1E1D288B1842288C308400801ED2
:1000400023288C1A45288C308400001C29280C1881
:1000500048288C308400801C2F288C184B282208BC
:1000600084002308F7002408F8002508F900260872
:10007000FA002708FB0020088A00210E8300FF0EEB
:100080007F0E09008A110A129A298A110A12802801
:100090008A110A1268298A110A1278290A108A100C
:1000A0000A11820730342E34313400340A108A1099
:1000B0000A1182075734443454340D340A3400345E
:1000C0000A108A100A11820743344F344D344D34DC
:1000D00041344E34443420344534523452344F3455
:1000E00052340D340A34003464008C1E742818080D
:1000F000EB001A08F800EB1C7F28181218160034C1
:10010000A0306E078400831303179D0104089C0030
:100110001D10831B1D140313742003171C08840077
:1001200083131D18831778088000A03003136E070F
:10013000840083130008243C031DA5280130EF0030
:10014000EE0124308316A0008312EF080319622900
:100150006E08043C031DC82804306E026D3EF80092
:10016000FA010318FA0A780803179B007A089C0022
:10017000A03003136E0784008313000803179D004B
:100180001B08840083131C1883171D0880000313A9
:100190000130EE076E08063C03186229EF01EE01FC
:1001A0000130EC00831621082F3C0318DB282108BE
:1001B000393C0318EB282108403C0318E3282108A8
:1001C000463C0318EB282108603C03181829210835
:1001D000663C031C182922082F3C0318F328220828
:1001E000393C031803292208403C0318FB28220845
:1001F000463C031803292208603C031818292208EA
:10020000663C031C18292208393C031809290930C7
:10021000A2070F30A2052108393C03181129093023
:10022000A1070F30A1050310210D2204F0001B29A6
:1002300083126916831625082F3C031823292508E5
:10024000393C031833292508403C03182B2925087D
:10025000463C031833292508603C0318602925080B
:10026000663C031C602926082F3C03183B292608FE
:10027000393C03184B292608403C0318432926081B
:10028000463C03184B292608603C031860292608C1
:10029000663C031C60292608393C031851290930A3
:1002A000A6070F30A6052508393C0318592909303F
:1002B000A5070F30A5050310250D2604F1006329BD
:1002C0008312E916831683128C128A110A122F28C0
:1002D000D50B74290130CD070318CE0A0319CF0AB4
:1002E0000319D00A0F30D5000C108A110A122F28DA
:1002F000D60B84290130D1070318D20A0319D30A77
:100300000319D40A6230D6008C108A110A122F28E1
:1003100083160C1083125008DA004F08D9004E08DB
:10032000D8004D08D70055080F3CDF0083160C1489
:1003300083120034691CA629E918A629E919A629FF
:1003400088210616831606128312E9148B108A116F
:100350000A122F288C1EAE297420AA298316861211
:10036000831286120034F21572088316870000305B
:100370008312871D0130F700770D8316C500C50D68
:10038000C50DF830C505721572088700003083125C
:10039000071D0130F700F70DF70DFC30F705770862
:1003A00083164504C700F2147208870000308312D8
:1003B000871C0130F7000310F70D770883164704F8
:1003C000C90072147208870000308312071C0130C4
:1003D000831649048312EA00AA21EC0183168C16C5
:1003E000C03083128B048A150A12832A7308840092
:1003F000831374188317031711088000840A80017F
:10040000F30A0319F40A031300340317901B222A7A
:100410000F30F700831603136F0EF7050A307702CB
:100420000318152A3030F7071B2A83120317100808
:10043000F70783160313770883120317910003133A
:10044000F62103170F3083160313EF050A306F02EE
:1004500003182C2A3030322A831203179013100805
:1004600083160313EF076F0883120317910003131A
:10047000F6210034031711089500100894001508A0
:10048000FA001408840083137A188317800803196C
:100490004D2A940A0319950A3F2A1308FA001208F4
:1004A000840083137A188317800803197C2A831623
:1004B00003136F08003C031C602A831203177C2A75
:1004C000831203171208840083131318831700087C
:1004D00098001408840083131518831718088000E7
:1004E000940A0319950A920A0319930A83160313AF
:1004F000EF03831203174D2A140884008313151881
:10050000831780011008F8001108F9000313003464
:1005100083168612831286160034882203179101EF
:1005200090011108013C031CB92A031D9B2A1008E5
:10053000903C031CB92AF217720883160313870034
:100540008312871BA82A031791019001AE2A031377
:1005500064001030F700F70BAB2A03178316031360
:10056000EF08031D640083120317900A0319910A10
:10057000912A0313AA2100340C1EBC2A0317180861
:10058000031399008A110A12FB2A1730840083177B
:1005900000080319DC2A0130F800BF30F7006400BE
:1005A000F70BCF2AF80BCD2A4A30F700F70BD62AE3
:1005B00000006400800BCB2A0034031716100313CD
:1005C0008822031793011308043C031C192B0313FF
:1005D0006B1303179401100814020318012B12085F
:1005E000FA0011088400831312188317000897007B
:1005F00098000313BC2A0317910A0319920A940A5C
:10060000EB2A03136B1B0F2B83166F088312031740
:1006100097000313C52203171614192B031383160F
:100620006F088312031797000313C5220317930A59
:10063000E32A0313AA210030031716180130F8002B
:1006400003130034F401C730F3003F300317910067
:100650000313F6216A088316EF005730831203173D
:100660009000031305222030031791000313F62195
:1006700003179101C73090008316031345088312B6
:100680000317930083160313440883120317920081
:10069000103083160313EF0083123A227908831671
:1006A000C5007808C400C6014608440784008313C7
:1006B00045188317800803195F2BC60A542BEF01D6
:1006C00083128D226A088316EF00460883120317EF
:1006D00090008316031345088312031792008316B4
:1006E000031344088312031791000313DD22F80853
:1006F000031D802B0A30031797000313C522622BBA
:1007000000348316C50803198D2B8312EC080319D6
:100710008B2B83168D2B812B83168312EC08031DE4
:10072000952B0030F800A52BA52B6A087002031D3D
:10073000A02B691AA02BEC010130F800A52BA52BEA
:100740006912EC010030F800A52B8A150A12F12A73
:1007500083164508FA004408840083137A18831727
:100760000008C8004708FA004608840083137A1876
:10077000831700084802031DD42B4508FA004408DB
:10078000840083137A1883178008031DCA2B003056
:10079000F800ED2B4508FA004408C40A0319C50AFD
:1007A000C60A0319C70AA92B4508FA0044088400A1
:1007B0008313451883170008C8004708FA00460845
:1007C0008400831347188317000848020318EB2B93
:1007D000FF30FA00EC2B0130F8008312003483164E
:1007E0000C108312D001CF01CE01CD010F30D50006
:1007F00083160C148C108312D401D301D201D101C1
:100800006230D60083168C148312061583160611E7
:1008100083120712721272088316870083128716DA
:10082000F212720883168700831269148A150A125D
:10083000052B20308316D000CC01CD01CE01CF0195
:100840004708FA004608F9004508F8004408F70090
:100850000310771C392C4808CC0749080318490FA6
:10086000CD074A0803184A0FCE074B0803184B0F51
:10087000CF07CF0CCE0CCD0CCC0CFA0CF90CF80C2D
:10088000F70CD00B282C831200348E30F70083161F
:100890004908F8004808F900FA01F808031D5A2C25
:1008A0007908F800F9010830F702F808031D5A2CFE
:1008B000F701622C0310F81B612CF90DF80DF703FA
:1008C0005A2CF81383120034831648080319D52CC8
:1008D000D0004C080319D52CD0070318762C7F3094
:1008E000D002031CD52C0319D52C7A2C8130D007CB
:1008F0000318D52C5008F700F801F901FA0149084E
:10090000D400D4174A08D3004B08D2001830D000C6
:10091000D101521CA32C4F08FA07031C952CF90A8D
:10092000031D952CF80A0319D1174E08F907031C6B
:100930009C2CF80A0319D1174D08CA00CA174A0897
:10094000F8070318D117D10DF80CF90CFA0CD40CD8
:10095000D30CD20C0310D00B882C0130F7070318EE
:10096000D52CF81BBA2CD40DFA0DF90DF80DF703A0
:100970000319D52CD41FCB2CFA0A031DCB2CF90A52
:10098000031DCB2CF80A031DCB2CF80CF90CFA0C28
:10099000F70A0319D52C4908D1004D08D106D11FFB
:1009A000D32CF817D92CF813D92CF701F801F90139
:1009B000FA0183120034B630F700FA01F901F801A8
:1009C00083164C084D044E044F04031DE92CF70117
:1009D000F62C0310F81BF52CCC0DCD0DCE0DCF0D44
:1009E000FA0DF90DF80DF70BE92CF813831200340A
:1009F0008030831CFE2C8316D10683128316D60109
:100A0000D7014D08D5005108D5064C080319EC2D27
:100A1000D400F70050080319F52DD4020319912DC5
:100A2000031C4F2D5108DA00DA175208D900530879
:100A3000D800D7010310DA0CD90CD80CD70CD40B82
:100A4000192DD51F262D5614092E56105410561642
:100A5000CF30840083131E2E5612D51B392D541C03
:100A6000442DDA0CD90CD80CD70CF70A0319042E34
:100A7000442DDA1B472D0310D70DD80DD90DDA0DF3
:100A8000F7030319042E392D5617B12D56134D08AF
:100A9000D500D51F4D2DDA17FD2DDA13FD2D500889
:100AA000D400F7004C08D4024D08DA00DA174E08DB
:100AB000D9004F08D800D7010310DA0CD90CD80C94
:100AC000D70CD40B5B2DD51F682DD614092ED6104C
:100AD0005410D616D330840083131E2ED612D51B85
:100AE0007B2D541C862DDA0CD90CD80CD70CF70AA8
:100AF0000319042E862DDA1B892D0310D70DD80D6E
:100B0000D90DDA0DF7030319042E7B2DD617B12D5D
:100B1000D6135108D500D51F8F2DDA17FD2DDA1306
:100B2000FD2D5108DA00DA175208D9005308D80011
:100B3000D51F9E2DDA135615092E5611D7015410C4
:100B4000CF30840083131E2ED51BC72D4D08D50032
:100B5000541CB12DDA0CD90CD80CD70CF70A031998
:100B6000042ED71FC22DD80A031DC22DD90A031D7A
:100B7000C22DDA0A031DC22DDA0CD90CD80CF70AE3
:100B80000319042E561B462DD61B882DE62D8030CA
:100B9000DA06DA1FCF2D092E5108D500DC2D4D08BD
:100BA000D500DA08031DDC2DD908031DDC2DD8087B
:100BB000031DDC2DF701FD2DDA1BE62D0310D70DEB
:100BC000D80DD90DDA0DF70BDC2D042ED51FEA2D2B
:100BD000DA17FD2DDA13FD2D5008F7005108DA0061
:100BE0005208D9005308D800FD2D4C08F7004D08D5
:100BF000DA004E08D9004F08D8005A08F800590802
:100C0000F9005808FA003C2EF701F801F901FA0141
:100C10003C2ED701D809D909DA09D709D70A031D0B
:100C2000172ED80A031D172ED90A0319DA0A5618E7
:100C3000252DD618672D56199D2DCC2D0008D807C7
:100C4000031C282ED90A031D282EDA0A031954146E
:100C500084030008D907031C302EDA0A0319541440
:100C600084030008801F803ADA0703185414561AC8
:100C70002C2DD61A6E2DA42D8312003483164C0809
:100C8000B63CCC00FA014D08D000CD170310CD0CB6
:100C9000CE0CCF0CFA0CF90CF80CF70CCC0B462E42
:100CA000D01F5D2EF709F809F909FA09F70A0319A7
:100CB000F80A0319F90A0319FA0A83120034F70132
:100CC000F801F901FA018316D801D901DA01DB0133
:100CD000570856045504540403199E2E2030DC0096
:100CE0000310D00DD10DD20DD30DD80DD90DDA0DC5
:100CF000DB0D57085B02031D872E56085A02031DA1
:100D0000872E55085902031D872E54085802031CCC
:100D1000982E5408D8025508031C550FD9025608BE
:100D2000031C560FDA025708031C570FDB0203148B
:100D3000F70DF80DF90DFA0DDC0B702ED83084008C
:100D400083138312003404088316C800C71FB52E0E
:100D5000C803C816C409C509C609C709C40A0319C6
:100D6000C50A0319C60A0319C70A3B30CF009A30D7
:100D7000CE00CA30CD00CC010A30CA004708D300EB
:100D80004608D2004508D1004408D0004F08D700DB
:100D90004E08D6004D08D5004C08D40083125F26BB
:100DA00000088316C400840A0008C500840A0008ED
:100DB000C600840A0008C700F708031DF22E4A087F
:100DC000013A0319F22E48080319F42E0F394A028A
:100DD0000319EC2E03181C2FC81B1C2F481BF42EC4
:100DE0002030142F2030C805C81E032FC8127708E2
:100DF000C8002D308312031791000313F6218316C8
:100E00004808F700C8013030C81E142FC8127708F0
:100E1000C8002D308312031791000313F6218316A7
:100E20004808F700C8013030F70777088312031726
:100E300091000313F62183164F08D3004E08D20009
:100E40004D08D1004C08D000D701D601D5010A3099
:100E5000D40083125F267A088316CF007908CE006B
:100E60007808CD007708CC00CA0BBE2E8312003460
:100E7000861483168610F401C730F3002A308312DB
:100E8000031791000313F6216A088316EF00573009
:100E90008312031790000313052203179101C73033
:100EA00090008316031345088312031793008316DB
:100EB00003134408831203179200103083160313A0
:100EC000EF0083123A2279088316C5007808C4001F
:100ED000C601460844078400831345188317800819
:100EE0000319742FC60A692FEF0183128D226A0835
:100EF0008316EF004608831203179000831603132E
:100F000045088312031792008316031344088312C3
:100F1000031791000313DD22F808031D952F0A30F3
:100F2000031797000313C522772F861083168610A8
:100F300083120034003069180130F700770D8316F2
:100F4000C500C50DFC30C50500308312691B01309A
:100F5000F7000310F70D770883164504C70000302B
:100F60008312E918013083164704F500F401393083
:100F7000F3007508EF005730831203179000031336
:100F800005220D30031791000313F6210A300317D1
:100F900091000313F6218316C5013930C400831272
:100FA00038278A150A12272BF4013930F3008316EB
:100FB000C401440883124E2000380319E92F831618
:100FC000C40A8312031791000313F6218316D92F45
:100FD00083120D30031791000313F6210A30031713
:100FE00091000313F6218316C5013930C400831222
:080FF00038278A150A12392B7B
:10100000691C8428E91C84285A088316C7008312A7
:1010100059088316C600831258088316C500831228
:1010200057088316C400CB01CA010330C900E83059
:10103000C8008A11831219248A157A088316C700FA
:101040007908C6007808C5007708C400C901831272
:101050005F088316C8008A11831245248A157A080E
:101060008316CB007908CA007808C9007708C80041
:101070004D30CF005530CE000530CD008530CC004E
:101080008A11831264248A1577088316C8007808A9
:10109000C9007908CA007A08CB004708CF00460883
:1010A000CE004508CD004408CC008A118312DB2411
:1010B0008A1583107A088316CF007908CE00780845
:1010C000CD007708CC004B08D3004A08D20049086D
:1010D000D1004808D0008A118312F8248A157A08B2
:1010E0008316CF007908CE007808CD007708CC00B1
:1010F0008A1183123E268A157A08E4007908E300F3
:101100007808E2007708E100F4013930F30041305B
:10111000840064088316C700831263088316C60020
:10112000831262088316C500831261088316C40007
:101130008A118312A3268A150D30031791008A1194
:101140000313F6218A150A30031791008A1103133D
:10115000F6218A158316C5013930C4008A1183121D
:1011600038278A158A150A12162BF4013930F30034
:101170004130840068088316C7008312670883160D
:10118000C600831266088316C5008312650883169D
:10119000C4008A118312A3268A150D30031791000B
:1011A0008A110313F6218A150A30031791008A1158
:1011B0000313F6218A158316C5013930C4008A113C
:1011C000831238278A158A150A124A2B8316440877
:1011D0000319AC29D00048080319AC29D002031C1C
:1011E000F6287F30D0070318AC29FC288130D002C4
:1011F000031CAC290319AC295008F700F801F901C8
:10120000FA01CF014508CE00CE174608CD004708A9
:10121000CC001930D0004B08CC0203181F29013034
:10122000CD0203181F29CE0203181F29CF0203186D
:101230001F29CF0ACE0ACD0A4B08CC0751294A08EC
:10124000CD0203183A290130CE0203183A29CF0201
:1012500003183A29CF0ACE0A4A08CD074B08CC0713
:10126000031C5129CD0A031D5129CE0A031D512902
:10127000CF0A512949088038CE020318502901307D
:10128000CF0203185029CF0A49088038CE074A08F0
:10129000CD07031C2E29CE0A031D2E29CF0A2E2985
:1012A0007A14D00B54295F290310CC0DCD0DCE0D2F
:1012B000CF0D0310FA0DF90DF80DD10D0B29511CAE
:1012C00067290310F80CF90CFA0CD10C6A29F70302
:1012D0000319AC29D11B93290310CC0DCD0DCE0DD4
:1012E000CF0D4B08CC0203187F290130CD02031823
:1012F0007F29CE0203187F29CF02031CA2294A08A6
:10130000CD0203188A290130CE0203188A29CF02A0
:10131000031CA22949088038CE0203189329013002
:10132000CF02031CA229FA0A031DA229F90A031DF0
:10133000A229F80A031DA229F70A0319AC29F80CFF
:10134000F90CFA0C4508D0004908D006D01FAA298C
:10135000F817B029F813B029F701F801F901FA01DB
:1013600083128A150A12AB2B83164508CC00490854
:10137000CC06CC1FC02903110310C51B0314F3298D
:101380004508CC004808CD004408CD020319CE29F9
:10139000CC1FF3290308013A8300F3294908CD0043
:1013A0004508CD020319DA29CC1FF3290308013AB5
:1013B0008300F3294A08CD004608CD020319E62927
:1013C000CC1FF3290308013A8300F3294B08CD0011
:1013D0004708CD020319F229CC1FF3290308013A6B
:1013E0008300F329031083128A150A12DD2B83165A
:1013F0008C1083125408DE005308DD005208DC0014
:101400005108DB005608623CE00083168C148312FE
:101410008A150A12E22B840183131F3083051930C9
:1014200083169900A6309800903083129800831696
:101430001F149F141F159F1107309C008312A901D0
:10144000AA014630AF00B0015130B100B2015330B3
:10145000B300B4015630B500B6014130B700B80151
:10146000CD01CE01CF01D001D101D201D301D401F0
:10147000D501D601D701D801D901DA01DB01DC01A0
:10148000DD01DE01DF01E001E101E201E301E40150
:10149000E501E601E701E8016910E9106911E911C8
:1014A0006912E9126913EA01EB01EF01FF30F00064
:1014B000F101F200F301F401F501F601FC01FD0177
:1014C000E9130F30D5006230D6000C30F70007303A
:1014D00081018130840083130008F03907388000CF
:1014E00064000008F739F719F03977048000853077
:1014F00090004830F80005389200FF3083169200C3
:101500008A118312B3298A150B1683160C148C14B6
:1015100083120716721272088316870083128712CD
:10152000F2127208831687008312861083168610C3
:1015300083120611831606118312061283160612F1
:101540001F1383121F179F1783169F1383121F14D5
:1015500083161F109F141F159F150030F80083126B
:101560001F08C73978049F0003081839F70083164D
:101570000E08033977040E148E14831503160B3AE4
:1015800083120319C72A133A0319E82AE92AF40136
:101590003930F3008316C40144088A11831256209F
:1015A0008A158316C40AF7008312031791008A1163
:1015B0000313F6218A15053083164402031DCC2A35
:1015C000C5013930C4008A11831222238A15E92A01
:1015D000E92A64006A088316C400C5018A118312CF
:1015E000812B8A15F80803196B2B8316C5016D3002
:1015F000C400C7012F30C6008A118312A8238A15A0
:10160000F808031D072B8A11EF2B8A156B2B831605
:10161000C5016D30C400C7013130C6008A11831284
:10162000A8238A15F808031D172B00286B2B831697
:10163000C5016D30C400C7013330C6008A11831262
:10164000A8238A15F808031D292B8A119A2F8A15B9
:101650006B2B8316C5016D30C400C7013530C60041
:101660008A118312A8238A15F808031D3B2B8A11BF
:10167000D42F8A156B2B8316C5016D30C400C701AA
:101680003730C6008A118312A8238A15F808031D73
:101690004B2BB5286B2BF4013930F3008316C401B2
:1016A00044088A11831260208A158316C40AF70041
:1016B0008312031791008A110313F6218A150F3044
:1016C00083164402031D502BC5013930C4008A1112
:1016D000831222238A15691C822BE918822BE919AF
:1016E000822B8A1188218A15DA08031D812BD908DB
:1016F000031D812BD808031D812B57081D3C03189F
:10170000822BE915691C642C6919642CE919642C75
:101710001F151F19892B1E088316C901C8008A11BD
:10172000831245248A157A088316C3007908C200FB
:101730007808C1007708C0004308C7004208C60007
:101740004108C5004008C400CB01CA01C901873067
:10175000C8008312E62877088316C4007808C500FD
:101760007908C6007A08C700CB004608CA004508B9
:10177000C9004408C800CF01CE012030CD0081301F
:10178000CC008A11831264248A157A088316C30058
:101790007908C2007808C1007708C000C701C601F7
:1017A000C5018030C4004308CB004208CA0041088C
:1017B000C9004008C8008312B4290318E12B031D97
:1017C000642CF7295E088316C70083125D08831610
:1017D000C60083125C088316C50083125B0883165B
:1017E000C400CB01CA010330C900E830C8008A1127
:1017F000831219248A157A088316C7007908C6004F
:101800007808C5007708C400C901831260088316F0
:10181000C8008A11831245248A157A088316CB00E2
:101820007908CA007808C9007708C8009630CF0048
:101830004330CE002330CD008230CC008A11831299
:1018400064248A1577088316C8007808C9007908C7
:10185000CA007A08CB004708CF004608CE004508EA
:10186000CD004408CC008A118312DB248A15831032
:101870007A088316CF007908CE007808CD00770863
:10188000CC004B08D3004A08D2004908D1004808D0
:10189000D0008A118312F8248A157A088316CF00A3
:1018A0007908CE007808CD007708CC008A11831221
:1018B0003E268A157A08E8007908E7007808E600ED
:1018C0007708E50069156917691C6A2CE9186A2C04
:0818D000E91D6A2CE92A6300FE
:02400E00753FFC
:00000001FF
